:020000040000FA
:060000005EEF10F012009B
:060800005EEF10F0120093
:0608080057EF0CF0120096
:06082A0001002421000082
:08083000000200002E00000090
:0808380058EC09F0FB0EDBCFC8
:10084000F3FFDB06F35000090AE0A6EC09F0FA0E0C
:1008500011EC0AF0F3E1151CF1E1010E01D0000EDC
:1008600087EF09F058EC09F03B0EE12402E3E16860
:10087000E652E16E010EDB6A020EDB6AF90EDBCF97
:10088000F6FFFA0EDBCFF7FFFB0EDBCFF8FF080019
:10089000F550DF6EDF5002E1ABEF08F0250EDF5CB4
:1008A00002E09EEF08F0030EDB6A040EDB6A050E21
:1008B000DB6A060EDB6A070EDB6AC0EC08F02D0E61
:1008C000DF5C0CE02B0EDF5C09E0200EDF5C06E055
:1008D000230EDF5C03E0300EDF5C1AE1DF50300AEC
:1008E00014E0130A0FE0030A0AE00B0A05E0060A07
:1008F000E4E1030EDB80E1D7030EDB82DED7030EDB
:10090000DB84DBD7030EDB86D8D7030EDB88D5D795
:100910002A0EDF5C1BE1BCEC08F00AEC09F010E0E9
:10092000030EDB8008680968130EDBCF0DF0140E90
:10093000DBCF0EF0BFEC0FF0040E06C0DBFF03D0E0
:10094000130EF3EC08F0C0EC08F00BD0090EDB6AD4
:1009500061EC09F003E0D5EC09F0FAD7090EF3ECED
:1009600008F0030EDBB0DB982E0EDF5C1BE1C0EC61
:1009700008F02A0EDF5C0BE1BCEC08F00AEC09F091
:1009800003E1130E45EC09F0C0EC08F00BD0090EA2
:10099000DB6A61EC09F003E0D5EC09F0FAD7090E47
:1009A00045EC09F0680EDF5C07E1C0EC08F0680E6A
:1009B000DF5C1DE1030E18D0740EDF5C17E07A0EC9
:1009C000DF5C14E0480EDF5C06E0540EDF5C03E001
:1009D0005A0EDF5C02E1020E07D06C0EDF5C03E012
:1009E0006A0EDF5C04E1010E98EC09F0C9DBDF5010
:1009F0006E0A01E17FD31E0A01E192D1200A01E1D2
:100A00008FD13F0A01E149D11A0A01E146D10D0A0D
:100A100001E143D1200A01E140D13A0A01E13DD18F
:100A2000200A01E13AD1260A01E135D10D0A01E19E
:100A300032D11A0A01E1D9D0200A4AE0300A1FE077
:100A4000460A0EE0250A01E083D3D950F90FE96E7A
:100A5000FF0EDA20EA6E010EEE5E000EEE5AEE5A3E
:100A6000A6EC09F0250EE66E95DB03E1151C01E10D
:100A700069D3A2EC09F001E26BD3DB2A69D3080E3B
:100A8000DB6A040EDB50010806E2040EDB046AECAC
:100A900009F0DB508BDB080EDB5009E0030EDB5066
:100AA000010B05E172DB01E04DD3080EDB6A64DB6C
:100AB000EFCFDFFF1AEC0AF003E1151C01E142D38E
:100AC000A2EC09F001E3DB2A60DB01E141D33AD378
:100AD000070EDB5002080FE1E6EC09F0030EADEC67
:100AE00009F00E0EEECFDBFF0F0EEECFDBFF100E88
:100AF000EECFDBFF20D0F70EDBCF17F0F80EDBCF09
:100B000018F0020E175E000E185AF70E17C0DBFF22
:100B1000F80E18C0DBFF17C0E9FF18C0EAFF9DEC14
:100B200009F0166A0E0E14C0DBFF0F0E15C0DBFFB6
:100B3000100E16C0DBFF0E0EDBCFE6FF0F0EDBCF75
:100B4000E6FF100EDBCFE6FF9AEC0FF0E552E55220
:100B5000E552130E07C0DBFF140E08C0DBFF060EC4
:100B6000DB5005E0130EE1EC09F001E26ADB05EC75
:100B70000AF002E2130E37DBC8EC09F006E0040EBF
:100B8000E1EC09F002E2050E2EDB030EDBB005D02E
:100B9000FCDA01E0D7D2080EDB6A090EDB6A0E0E22
:100BA000DBCFF6FF0F0EDBCFF7FF100EDBCFF8FF2A
:100BB0000800F550DF6EDF5014E00BEC0AF011E294
:100BC0001AEC0AF003E1151C01E1BCD2BBDB01E326
:100BD000DB2A090EDB2AD9500E0FE96E000ECBDBA3
:100BE000E7D7D3DA01E1B4D2ADD2C6DA110EEECF37
:100BF000DBFF120EEDCFDBFF110EDBCFE6FF120E97
:100C0000DBCFE6FF8CEC0FF0E552E552130EF3CF8D
:100C1000DBFF140EF4CFDBFF060EDB5004E0130EF7
:100C2000D0DB01E20EDB05EC0AF002E2130EDBDAA8
:100C3000AFDB05E0040EC5DB02E2050ED4DA030EDD
:100C4000DBB005D0A2DA01E07DD2080EDB6A090E26
:100C5000DB6A110EDBCFE9FF120EDBCFEAFFEFCF2D
:100C6000DFFFDF5014E0D7DB12E2E4DB03E1151C09
:100C700001E168D267DB01E3DB2A090EDB2A110EF2
:100C8000DB2ADBCFE9FF120EE8E3DB2AE6D77DDAC9
:100C900001E15ED257D2030EDB8E070EDB0410E1BA
:100CA00095DB040E5ADB0A0EEECFDBFF0B0EEECF08
:100CB000DBFF0C0EEECFDBFF0D0EEECFDBFF6CD0BB
:100CC000070EDB5003082CE1030EDBAE0DD0B2DAC9
:100CD000020E76DAEFCF14F0156A166A176A14AEB0
:100CE00039D01568166835D0F70EDBCF15F0F80E41
:100CF000DBCF16F0020E155E000E165AF70E15C069
:100D0000DBFFF80E16C0DBFF15C0E9FF16C0EAFFD7
:100D1000EFCF14F00A0E14C0DBFF0B0EDB6A38D0E5
:100D2000070EDB50020809E1030EDBAE04D059DBED
:100D300016AE10D00ED055DB0DD0030EDBAE12D0A8
:100D400079DA020E3DDAF9DA166A176A15AE02D0C0
:100D500016681768E2DA0C0E16C0DBFF0D0E17C01E
:100D6000DBFF1AD0F70EDBCF16F0F80EDBCF17F053
:100D7000020E165E000E175AF70E16C0DBFFF80EB5
:100D800017C0DBFF16C0E9FF17C0EAFFD6DAC5DAE5
:100D90000C0EDB6A0D0EDB6A060EDB5005E1010E60
:100DA000F36E050EF3CFDBFF150EDB6A160EDB6A62
:100DB000D950370F146E000EDA20156E390E14C09C
:100DC000DBFF3A0E15C0DBFF380EDB6A080EDB6A6C
:100DD0000A0EAEDADF50780A12E0200A10E0280A84
:100DE0000CE0200A0AE03F0A06E00D0A02E0200AB1
:100DF00008E1020E05D0080E03D0080EDF26100E03
:100E000097DA030EDBBE02D0DB92DB94DB50800B63
:100E100024E08ADAD890030EEB50000A08E6000EB0
:100E2000EE5C000EEE58000EEE58000EEE5815E285
:100E300013DA0B680C680D680E6854EC0FF00A0E9C
:100E400002C0DBFF0B0E03C0DBFF0C0E04C0DBFF98
:100E50000D0E05C0DBFF2D0E08D0030EDBA202D065
:100E60002B0E03D0DBA408D0200EF36E170EF3CFA9
:100E7000DBFF150EDB2A02D0170EDB6A050EDB50F6
:100E800003E1B7D901E189D00A0E146E210E156E67
:100E9000000E166E070EDBCF17F0186A196A1A6A71
:100EA00017C00BF018C00CF019C00DF01AC00EF0EE
:100EB000D3D9ECEC0FF014500224F36E155003203C
:100EC000F46E16500420F86EF4CFF7FFF3CFF6FF60
:100ED0000800090EF5CFDBFF580EDF5C0FE1610E55
:100EE000F36E090E7BD90AE3200E146E090EDBCFD8
:100EF000E7FF1450E75E090EE7CFDBFF070EDBCFFD
:100F000014F0156A166A176A0FDA14C00BF015C0D0
:100F10000CF016C00DF017C00EF0EECF06F0EECFBD
:100F200007F0EECF08F0EFCF09F0ECEC0FF009C0BE
:100F3000EDFF08C0EDFF07C0EDFF06C0EFFF390E63
:100F4000DBCFE9FFDB063A0EDBCFEAFF01E2DB068F
:100F5000090EDBCFEFFF150EDB2A4BD995E1030E0F
:100F6000DBA61DD06F0EDF5C06E1C1D918E3150EBC
:100F7000DB285BDA14D0780EDF5C09E0580EDF5C0A
:100F800006E0620EDF5C03E0420EDF5C08E1020E69
:100F9000F36E160EF3CFDBFF02D0150EDB6A030EE5
:100FA000DB50100B0EE0040EDBCF14F0050EDB500F
:100FB000D880145406E2060EDB5003E1040EDB5029
:100FC00034DA95D90AE2050EDBCFE7FF150EDB50C8
:100FD000E75E050EE7CFDBFF02D0050EDB6A040EED
:100FE000DBCF14F0160E45D9D880145414E2160E37
:100FF000DBCFE6FF150EDBCFE6FF040EDBCFE6FF0F
:10100000050EDB50E552E75CE552D880E754E55227
:10101000D880E7545FD9030EDB50010B0BE1080EBB
:10102000DB5008E0B2D801E08DD0080EDB50BED80E
:10103000080EDB6A170EDB5007E088D9170EF1D9CE
:1010400003E1151C01E17ED0160EDB5016E07ED9BF
:10105000300EE66E9FD802E1151C74E077D9DFCF21
:10106000E6FF12EC0FF0E552E552E552F4CF15F031
:101070000001F31C02E1151C65E0050EDBCF14F046
:10108000160EDB50D880145409E2050EDBCFE7FFC3
:10109000160EDB50E75E050EE7CFDBFF300EE66E87
:1010A000050ECBD94FE1390EDB2ADBCFE9FF3A0E33
:1010B00001E3DB2ADBCFEAFF090EEFCFDBFFDB50DA
:1010C0000EE044D9090EADD902E1151C3BE0390E02
:1010D000DB2ADBCFE9FF3A0EEDE3DB2AEBD755D86D
:1010E00031E1160EDBCFE6FF080EC3D8E552E72448
:1010F0005DD82ED0070EDB50030A1CE0010A14E075
:10110000030A07E07BD9DBCFEEFF020EDBCFEDFF5A
:101110001FD0F5D8196A17AE02D0186819682CD8F4
:10112000BCD819C0EEFF14D0EAD817BE186824D86E
:10113000B4D80ED063D9DBCFEFFF0AD07BD905E15D
:10114000151C03E1F368F46810D0FCD801E3DB2A36
:1011500079D947EF04F0010EDBCF14F0020EDBCF9C
:1011600015F014C0F3FF15C0F4FF3B0EE15C02E282
:10117000E16AE552E16ECBD029D9020EADEF09F05C
:1011800061D90800F550DF6E1200200EE66E080EE1
:101190001DEF0AF012EC0FF0E552E552E552F3CFE5
:1011A00014F0F4CF15F00001F31C1200146E156A50
:1011B000D950010F4DD91450EE261550ED221200D2
:1011C000185E000E195AF70E18C0DBFFF80E19C092
:1011D000DBFF18C0E9FF19C0EAFF1200DBCFF4FF04
:1011E000F350F45C1200DB50E76E040EE7CFDBFF38
:1011F00012000A0EDBCF14F00B0EDBCF15F00C0E35
:10120000DBCF16F00D0EDBCF17F0145015101610B3
:1012100017101200130EEECFDBFF140EEDCFDBFF25
:10122000130EDBCF14F0140EDBCF15F00001800E8F
:1012300015141200F70EDBCF18F0F80EDBCF19F003
:101240001200050EDB50E66ED950130F01D9E5529E
:10125000E750EE6EED6A12000A0EDBCF06F00B0EC1
:10126000DBCF07F00C0EDBCF08F00D0EDBCF09F063
:101270001200DBCFE6FF150EDBCFE6FF050EDB50DD
:10128000E552E724E552E7241200DB50CED8010EE8
:10129000F36E060EF3CFDBFF1200EE50EFCFEAFF46
:1012A000E96E16C0EEFF17C0EEFF18C0EEFF120089
:1012B000D9CFE6FFDACFE6FFE1CFD9FFE2CFDAFF01
:1012C0001200DFCFE6FFE66A2CEC10F0E552E552A3
:1012D000F3501200E76E080EE7CFDBFF1200EECFEF
:1012E00014F0EECF15F0EFCF16F0176A1200050ECE
:1012F000DBCF14F0150EDB50D88014541200010E11
:10130000DBCF16F0020EDBCF17F0186A1200E552A1
:10131000E5CFDAFFE7CFD9FF12000A0E14C0DBFFDA
:101320000B0E15C0DBFF1200D9500A0F28EF0AF090
:10133000F36E070EF3CFDBFF1200EECF14F0EFCF0A
:1013400015F01200010EDB2A020E1200FC0EDBCF9C
:10135000E6FFFD0EDBCFE6FF1200145E000E155A0D
:10136000F70E14C0DBFFF80E15C0DBFF14C0E9FF59
:1013700015C0EAFF1200DA20EA6EEF2AEECFF6FF80
:10138000000EEF22EECFF7FFEF22EECFF8FF1200B4
:10139000040EDBCFE6FF130EDB50E552E75C9ADF6D
:1013A000DB5004DF060EDB501200090EDB500A0D85
:1013B000F350DF24D00FE76E090EE7CFDBFFC0EF5D
:1013C00008F0DB50F36E050EEEEF08F0F70EDBCF02
:1013D00014F0F80EDBCF15F01200DFCFE6FFCAEFF6
:1013E00008F028DF030EECDE6FEF09F01CEC04F0D0
:1013F000E552E552E552E55200091200BDDEEE501D
:10140000EFCFEAFFE96E010E1200130EDB50F36E10
:10141000040EEEEF08F0040EDB50F36E090EEEEF53
:1014200008F0DBCFE6FFCAEF08F0E76E050EE7CF66
:10143000DBFF12008BDFEDEF09F0DBCFE6FF86DF8D
:10144000F6EF09F0D950F90FE96EFF0EBBEF09F086
:0A145000E96E000EDA20EA6E1200C9
:06145A00D9CFE6FFE1CF4F
:10146000D9FF040EE126DE6ADE6ADE6ADD6ADD523D
:10147000DD52FD0EDBCF14F0FE0EDBCF15F0166A49
:10148000176A15AE02D016681768D9CFE9FFDACF10
:10149000EAFF030EEB501718E8AE02D0173408D05D
:1014A0001450EE5C1550EE581650EE581750EE588A
:1014B0000FE20C0EE66E3EEC10F0E552D9CFE9FFDC
:1014C000DACFEAFFEE2A000EEE22EE22EE22D1D78C
:1014D000040EE15C02E2E16AE552E16EE552E7CF1B
:1014E000D9FF12000F0EC16E070EB46E936A300E54
:1014F000926E0F0E946EF19E1200D9CFE6FFE1CFEF
:10150000D9FF020EE1268250020B01E0010E080D08
:10151000F3CF16F08250010B040DF3CF15F080507D
:10152000200B01E0010EE824146E8050100B01E046
:10153000010E142415241624DE6EDD6ADECF14F0AD
:10154000DDCF15F014C0F3FF15C0F4FF020EE15C0F
:1015500003E200D0E16AE552E16EE552E7CFD9FF40
:1015600012008092320EE66E7AEC10F0E552808422
:10157000320EE66E7AEC10F0E5528094320EE66E92
:101580007AEC10F0E55212008082320EE66E7AECB0
:1015900010F0E5528084320EE66E7AEC10F0E552DF
:1015A0008094320EE66E7AEC10F0E5521200380E9E
:1015B000816ED7DF320EE66EE66A4FDFE552E55206
:1015C000010E816ECEDF320EE66EE66A46DFE55230
:1015D000E5520D0E816EC5DF320EE66EE66A3DDF26
:1015E000E552E552060E816EBCDF320EE66EE66A0B
:1015F00034DFE552E5521200010E816EB2DF0A0EB1
:10160000E66EE66A2ADFE552E5521200D9CFE6FF20
:10161000E1CFD9FF020E816EA4DF0A0EE66EE66A04
:101620001CDFE552E552FD0EDBCFE6FFFE0EDB5080
:10163000280DF350E552E724E76EFE0EE7CFDBFFFF
:10164000FD0EDB6AFE0EDB50F36EFD0EDBCFF4FF0A
:10165000F350F45C0BE2140E816E83DF320EE66E03
:101660007AEC10F0E552FD0EDB2AECD7E552E7CF1D
:10167000D9FF1200D9CFE6FFE1CFD9FFFE0EDB5034
:10168000816E82DF320EE66E7AEC10F0E552E552A2
:10169000E7CFD9FF1200D9CFE6FFE1CFD9FFFD0E8A
:1016A000DBCFE9FFFE0EDBCFEAFFEF500EE0FD0ED1
:1016B000DBCFE9FFDB2AFE0EDBCFEAFF01E3DB2A0B
:1016C000EF50E66ED7DFE552EAD7E552E7CFD9FF14
:1016D00012000001646B300E926EF00E936EEF0EEE
:1016E000606F60C081FF040E616F6151000821E2EC
:1016F0006051FE0BE842606F60C081FF050EE66E30
:10170000E66AABDEE552E5528150100B09E08150EC
:10171000200B06E08150400B03E08150800B01E17B
:101720000AD80001640502E1655104D06105616FCA
:10173000DCD7CFD71200F00E936E81CF63F000019B
:101740006315626F0F0E6015606F60516211606FFC
:1017500081CF63F0F00E6315626FF00E625D01E001
:10176000F7D7936A06D866C065F00001010E646F72
:1017700012000001676B100E675D14E26751EA6AA0
:10178000000FE96E020EEA22EF50605D08E167513A
:10179000EA6A100FE96E020EEA22EFCF66F06729BF
:1017A000676FE9D766C081FF640EE66EE66A55DEB4
:1017B000E552E55212000001686B070E685D1DE2FC
:1017C00088DF0001696F6851EA6A6A0FE96E000EEE
:1017D000EA2269C0EFFF6851EA6A6A0FE96E000EFB
:1017E000EA22EF50460802E108D004D069C0E6FFC3
:1017F00041DFE5520001682BE0D76851EA6A6A0FC1
:10180000E96E000EEA22EF6A12000001686B070E13
:10181000685D16E26851EA6A6A0FE96E000EEA2214
:10182000EF50E66E27DFE55200016829EA6A6A0F89
:10183000E96E000EEA22EF5001E102D0682BE7D7F3
:101840001200D9CFE6FFE1CFD9FFE652F250800B6C
:1018500001E0010EDF6EF29EA69EA69CA684FE0EFF
:10186000DB50A96EFD0EDB50A86E550EA76EAA0EBA
:10187000A76EA682A6B2FED7A694DF50E8B0F28E7D
:10188000E8A0F29EE552E552E7CFD9FF1200D9CF8A
:10189000E6FFE1CFD9FFA69CA69EFE0EDB50A96E07
:1018A000A680A85000D0E552E7CFD9FF1200DACFCA
:1018B000E4FFE2CFDAFFE65200017507000E765B27
:1018C000D8907651000A08E6000E735D000E745938
:1018D000010E7559000E765909E21B0E7427B70EDA
:1018E0007523000E76230201202B212302013C0EDA
:1018F000201901E1215119E12C2B000E2D23206B21
:10190000216B3C0E2C1901E12D510FE12A2B000E09
:101910002B232C6B2D6B180E2A1901E12B5105E19D
:10192000282B000E29232A6B2B6BF294E552E5CF6E
:10193000DAFF1100D7DD816AEBD80001736B1B0E53
:10194000746FB70E756F766B9F0EE66E10EC10F02D
:10195000E552F28E0ED802012251201902E12351E4
:10196000211905E020C222F221C223F24DD8F3D77B
:101970001200D9CFE6FFE1CFD9FF100EE126D9CF73
:10198000E9FFDACFEAFF480EEE6E4F0EEE6E520E12
:10199000EE6E410EEE6E3A0EEE6EEE6AD950060F06
:1019A000E96EDACFEAFF300EEE6EEE6E3A0EEE6EB4
:1019B000300EEE6EEE6E3A0EEE6E300EEE6EEE6E97
:1019C000EE6AEE6AF4DD18DED9CFE6FFDACFE6FF85
:1019D00062DEE552E552E66A010EE66E17DEE5527A
:1019E000E552D950060FE66E000EDA20E66E53DEA1
:1019F000E552E552100EE15C02E2E16AE552E16E69
:101A0000E552E7CFD9FF1200D9CFE6FFE1CFD9FFEA
:101A10000A0EE126E66A010EE66EF8DDE552E552B1
:101A20002AC2E6FF2BC2E6FF1B0E146E210E156EB6
:101A3000166A14C0E6FF15C0E6FF16C0E6FFD9CF50
:101A4000E6FFDACFE6FF6DEC0EF0176E070EE15EF3
:101A50001750D9CFE6FFDACFE6FF1DDEE552E5529B
:101A6000030EE66E010EE66ED1DDE552E5522CC2A4
:101A7000E6FF2DC2E6FF1B0E146E210E156E166AD0
:101A800014C0E6FF15C0E6FF16C0E6FFD9CFE6FF9B
:101A9000DACFE6FF6DEC0EF0176E070EE15E175021
:101AA000D9CFE6FFDACFE6FFF6DDE552E552060EC6
:101AB000E66E010EE66EAADDE552E55220C2E6FFB3
:101AC00021C2E6FF1B0E146E210E156E166A14C09D
:101AD000E6FF15C0E6FF16C0E6FFD9CFE6FFDACF76
:101AE000E6FF6DEC0EF0176E070EE15E1750D9CFD2
:101AF000E6FFDACFE6FFCFDDE552E5520A0EE15C04
:101B000002E2E16AE552E16EE552E7CFD9FF120049
:101B1000D9CFE6FFE1CFD9FF080EE126D950030F58
:101B2000E96EDACFEAFF530EEE6E450EEE6E540EFE
:101B3000EE6E3E0EEE6EEE6A3ADD5EDDD950030FBC
:101B4000E66E000EDA20E66EA6DDE552E552E66AA4
:101B5000010EE66E5BDDE552E5522DDEE66A010E12
:101B6000E66E54DDE552E55250DE6AC0DFFF010E3D
:101B70006BC0DBFF020EDB6AD9CFE6FFDACFE6FFF0
:101B8000F8EC0DF0E552E552F3CF2AF2F4CF2BF248
:101B90006CC0DFFF010E6DC0DBFF020EDB6AD9CF28
:101BA000E6FFDACFE6FFF8EC0DF0E552E552F3CFB1
:101BB0002CF2F4CF2DF26EC0DFFF010E6FC0DBFF01
:101BC000020EDB6AD9CFE6FFDACFE6FFF8EC0DF0C4
:101BD000E552E552F3CF20F2F4CF21F2080EE15C9A
:101BE00002E2E16AE552E16EE552E7CFD9FF120069
:101BF000FF0EE3CFEAFFE552FF0EE3CFE9FFE55228
:101C0000E66AE66AD9CFE6FFDACFE6FFFC0EE1240A
:101C1000D96EFF0EE220DA6EE66AE66AE66A200E08
:101C2000EF5C06E0090EEF5C03E0EF6603D03FD007
:101C3000EE50F5D72D0EEF5C03E1FF0EE32A03D043
:101C40002B0EEF5C01E1EE502F0EEF6424D03A0E24
:101C5000EF6021D0D890F90EE336FA0EE336FD0E90
:101C6000DECFE3FFFE0EDDCFE3FFD890F90EE336C3
:101C7000FA0EE336D890F90EE336FA0EE336FD0E8F
:101C8000E350DE26FE0EE350DD22300EEE5CDE2653
:101C9000000EDD22D9D7FF0EE3CFE8FFE85207E0C0
:101CA000F90EE31EE32AFA0ED8B4E306E31EE5526A
:101CB000E552E552FF0EE3CFDAFFE552FF0EE3CF28
:101CC000D9FFE552E1CFE9FFE2CFEAFFED52ED5255
:0A1CD000EECFF3FFEFCFF4FF120098
:061CDA00D9CFE6FFDACFCE
:101CE000E6FFE1CFD9FFE2CFDAFFE652E652E65255
:101CF000E652D950F90F146EFF0EDA20156E020E5F
:101D000014C0DBFF030E15C0DBFF020EDBCFE6FFC6
:101D1000030EDBCFE6FFF90EDBCFE6FFFA0EDBCFDB
:101D2000E6FFFB0EDBCFE6FFD950FC0FE66EFF0EA1
:101D3000DA20E66E32EC04F0146E070EE15C02E28B
:101D4000E16AE552E16E1450F3CFDEFFF4CFDDFF20
:101D5000FC0EDBCFE9FFFD0EDBCFEAFFEF6ADECF43
:101D600014F0DDCF15F014C0F3FF15C0F4FF040E1E
:101D7000E15C02E2E16AE552E16EE552E5CFDAFFAD
:061D8000E7CFD9FF1200BD
:0A1D86002A0EF66E080EF76E000E2E
:101D9000F86E02010900F550336F0900F550346FF9
:101DA00003E1336701D03DD00900F5502E6F0900E3
:101DB000F5502F6F0900F550306F09000900F550FC
:101DC000E96E0900F550EA6E090009000900F550B6
:101DD000316F0900F550326F09000900F6CF35F276
:101DE000F7CF36F2F8CF37F22EC2F6FF2FC2F7FF49
:101DF00030C2F8FF0201315302E1325307E009001B
:101E0000F550EE6E3107F8E23207F9D735C2F6FF2A
:101E100036C2F7FF37C2F8FF02013307000E345B0A
:041E2000BFD7120016
:0C1E2400D9CFE6FFDACFE6FFE1CFD9FF0F
:101E3000E2CFDAFFFB0EDBCF14F0FC0EDBCF15F0A8
:101E40000001800E15141AE1FB0EDBCFE9FFFC0E3A
:101E5000DBCFEAFFEECFF3FFEDCFF4FFEE2A000E6B
:101E6000EF22F3CFE9FFF4CFEAFFFD0EDBCFEFFF68
:101E7000EF50156AF36E15C0F4FF10D0FB0EDB5067
:101E8000FE0806E1FD0EDBCFE6FF6CEC10F005D09E
:101E9000FD0EDBCFE6FF90EC10F0E552E552E5CF0A
:081EA000DAFFE7CFD9FF1200C1
:081EA80006500B02F3CF02F01B
:101EB000F4CF03F00C02F3500326000EF420046E5E
:101EC00006500D02F3500426000EF420056E065055
:101ED0000E02F350052607500B02F3500326F45070
:101EE0000422000E052207500C02F3500426F45081
:101EF000052207500D02F350052608500B02F3503F
:101F00000426F450052208500C02F350052609500F
:081F10000B02F350052612003C
:081F1800FE0EE3CFE9FFFF0E0E
:101F2000E3CFEAFFF36AF46AEE5203E0F34AF42ADD
:101F3000FBD71200FF0EE3CFF8FFE552FF0EE3CF11
:101F4000F7FFE552FF0EE3CFF6FFE552E66AE66AD9
:101F5000E66A0900F55209E0FD0EE32A05E1FE0EEE
:101F6000E32A02E1FF0EE32AF4D7FD0EE3CF07F0E8
:0E1F7000FE0EE3CF08F0FF0EE3CF09F01200E3
:021F7E0009C098
:101F800013F008C012F008500D02F4CF07F0F3CFA1
:101F900006F009500E02F4CF09F0F3CF08F00D025D
:101FA000F3500726F4500822E86A092212500E0264
:101FB000F3500726F4500822E86A09220EAEE5EF36
:101FC0000FF01250085E1350095A13AE000C0D505A
:081FD000085E0E50095A000CD6
:081FD800056A046A036A026A4B
:101FE000200EE76ED89006360736083609360236D8
:101FF0000336043605360B50025C0C5003580D5066
:1020000004580E50055809E30B50025E0C50035A59
:102010000D50045A0E50055A062AE72EE4D7120036
:10202000D9CFE6FFDACFE6FFE1CFD9FFE2CFDAFF83
:10203000FD0EDB507F0BD56ED76AD66AF294FD0E8B
:10204000DBAE02D0F28A01D0F29AD58EE552E5CF0E
:08205000DAFFE7CFD9FF12000F
:08205800F36AF46AFF0EE124B3
:10206000E96EFF0EE220EA6EED6607D02F0EEF64F8
:0C20700004D03A0EEF6001D0F32A1200F9
:04207C00FF0EE35020
:102080001B6E480E01D04C0EE76EE72EFED7E76AB6
:0C209000E72EFED71B2EF7D70000120031
:04209C00000EF36ED1
:1020A00000EE00F0080E01D81200EA6002D0EE6ADD
:0C20B000FCD7F350E9601200EE6AFCD788
:0420BC0012EE40F0F0
:1020C00022EE40F0F86A019CC3EC0EF091EC10F0A7
:0820D0009AEC0CF0FBD71200A2
:0820D800FF0EE350ACBA04D086
:1020E000AF6AAB8EAC8A949CACA2FED7AD6EF36E99
:0420F000F46A12007C
:0C20F400FF0EE350E84E1200000000D088
:0A21000000D000D0E82EFAD712003C
:06210A00303132333435A0
:0B211000363738396162636465660091
:05211B002530327500C3
:022120001200AB
:022122001200A9
:0C212400EEEDEBE7DEDDDBD7BEBDBBB7A8
:102130007E7D7B7730313233343536373839414222
:10214000434445460000000000000000000000007D
:0221500000008D
:00000001FF
